:100000000C9434000C9446000C9446000C9446006A
:100010000C9446000C9446000C9446000C94460048
:100020000C9446000C9446000C9446000C94460038
:100030000C9446000C9446000C9448000C94460026
:100040000C9446000C9446000C9446000C94460018
:100050000C9446000C9446000C9446000C94460008
:100060000C9446000C94460011241FBECFEFD8E03C
:10007000DEBFCDBF11E0A0E0B1E001C01D92A23013
:10008000B107E1F70E9463000C94AC010C940000EE
:100090001F920F920FB60F9211248F93809100013F
:1000A0008F5F80930001809101018F5F8093010138
:1000B0008A3019F488B18F7C88B98F910F900FBE68
:1000C0000F901F9018958FEC8093640014B880EE09
:1000D00085B99FE397B918B88AB98FE18BB982E0E7
:1000E00084BD94E095BD9CE797BD80936E007894A5
:1000F000E0E070E0F0E080E030E020E090E04FEF02
:10010000BFEF1DC0452F6623D9F0509100015E312D
:10011000B8F0FF23A1F04D9B06C0992309F4419844
:10012000222369F407C04E9B07C0332309F441988A
:10013000882329F4439803C058B1557F58B960E02B
:1001400059B15F715F3171F15B1761F15B3109F496
:10015000FDC05C3128F45F30C1F0573171F408C044
:100160005D3119F05E3149F4EDC080E031E002C04C
:1001700081E030E020E091E0EDC0FF2359F04D9B9D
:1001800009C04E9B07C05E9805C0F0E081E030E0FA
:1001900020E091E0A8B1AA7FA8B9A8B1A57FA8B92D
:1001A000406FB52F4F9B1CC01C9B2EC059B1507681
:1001B000A1F04D9B04C09111419A2111439A4E9B8D
:1001C00004C03111419A8111439A1D9B06C01092BF
:1001D0000001509100015E31E0F35F98406F14C060
:1001E0001C9912C05F9A56B15A7071F058B15A7F7B
:1001F00058B91D9B06C010920001509100015E315C
:10020000E0F358B1557F58B9A3B15A2F5F70541716
:1002100009F479CFA1FF0CC04D9B09C05D989923CB
:1002200011F040984198222311F04298439870E0D1
:10023000452F487061F04E9B09C05E98332311F042
:1002400040984198882311F042984398E0E0452F68
:1002500051FD29C04D9927C0FF23F1F04E9B1CC0D2
:10026000109201011E9913C0A8B1AA7FA8B95E9887
:10027000EE2391F4459A1D9B05C010920001E1E028
:1002800061E00AC0E8B1E57FE8B9E1E005C07723A5
:1002900051F4449A71E007C05D9A4F9904C09111DE
:1002A000419A2111439A43FD29C04E9927C0FF234B
:1002B000F1F04D9B1CC0109201011F9913C0A8B111
:1002C000AA7FA8B95D98772391F4449A1D9B05C035
:1002D0001092000171E061E00AC078B1757F78B9D1
:1002E00071E005C0EE2351F4459AE1E007C05E9A43
:1002F0004F9904C03111419A8111439A4F9902CF0D
:100300004D9B0CC040FF06C091114098222331F054
:10031000429804C09111409A2111429A4E9BF2CE0C
:1003200042FF07C031114098882309F4EBCE429870
:1003300006C03111409A882309F4E4CE429A452F31
:1003400081E0E1CE81E031E021E015CF81E030E0D5
:0C03500021E090E0F1E013CFF894FFCF23
:00000001FF
